:020000040800F2
:107000001817002099710008417F0008317E0008A0
:107010003D7F0008197A00089988000800000000E8
:107020000000000000000000000000005583000880
:10703000157C000800000000AF710008B171000865
:10704000B3710008B3710008B371000841820008F1
:10705000B3710008B3710008B3710008B371000880
:10706000B3710008B3710008B3710008B371000870
:10707000B3710008B3710008B3710008B371000860
:10708000B3710008B3710008B3710008B371000850
:10709000B3710008B3710008B3710008B371000840
:1070A000B3710008B3710008B3710008B371000830
:1070B000B3710008C9840008B3710008B3710008F7
:1070C000B3710008B3710008B3710008B371000810
:1070D000B371000895860008B3710008B371000809
:1070E000B3710008B3710008B371000800F002F832
:1070F00000F042F80AA090E8000C82448344AAF110
:107100000107DA4501D100F037F8AFF2090EBAE80D
:107110000F0013F0010F18BFFB1A43F001031847CB
:10712000B45F0000D45F0000103A24BF78C878C173
:10713000FAD8520724BF30C830C144BF04680C607D
:10714000704700000023002400250026103A28BFC5
:1071500078C1FBD8520728BF30C148BF0B607047C9
:10716000642900F09D80732900F08F820020704711
:107170001FB51FBD10B510BD00F0BDFA1146FFF7D9
:10718000F7FF02F0BBFC00F0DBFA03B4FFF7F2FFFD
:1071900003BC00F0E5FA00000948804709480047B1
:1071A000FEE7FEE7FEE7FEE7FEE7FEE7FEE7FEE7B7
:1071B000FEE7FEE704480549054A064B7047000014
:1071C00069840008ED7000081805002018170020D9
:1071D00018070020180700200FB41CB5074B06AA9B
:1071E0007B4469460090059800F025FA0020694626
:1071F00000F034FA1CBC5DF814FB000079040000B8
:1072000070B5044685690068C10601D5302600E0E6
:107210002026C00707D070BDD4E901213046904731
:10722000206A401C20626D1EF6D570BD70B5044604
:1072300085690078C00707D170BDD4E901212020FD
:107240009047206A401C20626D1EF6D570BD70B557
:107250000C460546012A05D02878800600D5EA6943
:10726000002302E0012305E05B1C934202D2E05CB4
:107270000028F9D1A869E618C01AA861286A18443C
:1072800028622846FFF7BCFF04E0D5E9012114F885
:10729000010B9047B442F8D32846FFF7C7FF70BDF3
:1072A0002DE9F0410646002410687529314616A5DF
:1072B00010D0AFF30080002802DA404213A507E0A7
:1072C00031688A0701D512A502E0490704D511A546
:1072D000012401E0AFF3008000210A2206F1240717
:1072E00009E0B0FBF2FCB0FBF2F302FB1C00303013
:1072F00078541846491C0028F3D123462A463046C4
:10730000BDE8F04100F039B9000000002D00000098
:107310002B000000200000002DE9F0474FF0000A8C
:1073200089460446C0F820A02046E1688847002826
:1073300076D0252806D0D4E901219047206A401C48
:107340002062F1E7E168204600258847C4F81CA0C8
:1073500006460027C4F818A02A2E09D0304601F0AE
:107360009DFA38B304EB8708303EC8F8186019E07E
:1073700059F8041B204604EB87029161E1688847B5
:10738000012F064618D1E069002820DA25F02005F3
:107390001DE0D8F8180000EB800006EB4000303804
:1073A000C8F818002046E1688847064601F076FADA
:1073B0000028EED1012F0AD02E2E08D12046E168F8
:1073C00088477F1C0646022F45F02005C4DBA069D4
:1073D000002803DA404245F00105A061E80701D02A
:1073E00025F01005B6B1A6F14100192802D82036C3
:1073F00045F400654A463146204625604D46FFF774
:10740000AFFE58B1012806D0ED1D25F0070000F1B0
:10741000080989E704E005F1040985E730468AE7B1
:10742000206ABDE8F08730B505460B462A4613F8BA
:10743000014B12F8010B08B1A042F8D01CB1002892
:1074400002D06D1CF1E7284630BD40EA010310B5BB
:107450009B070FD1042A0DD310C808C9121F9C42E4
:10746000F8D020BA19BA884201D9012010BD4FF0D6
:10747000FF3010BD1AB1D30703D0521C07E0002023
:1074800010BD10F8013B11F8014B1B1B07D110F880
:10749000013B11F8014B1B1B01D1921EF1D1184683
:1074A00010BD40EA0103024630B59B0710D14FF0F2
:1074B000013400E008C208C91D1B9D4315EAC41F22
:1074C000F8D013F0FF0102F8011B0DD01B0AF8E7FA
:1074D00011F8013B002B02F8013B05D011F8013BEC
:1074E000002B02F8013BF3D130BD032A40F230807B
:1074F00010F0030C00F0158011F8013BBCF1020FF5
:10750000624498BF11F801CB00F8013B38BF11F875
:10751000013BA2F1040298BF00F801CB38BF00F88C
:10752000013B11F0030300F0B480083AC0F008807A
:1075300051F8043B083A51F804CBA0E80810F5E7ED
:10754000121D5CBF51F8043B40F8043BAFF30080D0
:10755000D20724BF11F8013B11F801CB48BF11F845
:10756000012B24BF00F8013B00F801CB48BF00F815
:10757000012B70477047704770472DE9F0470D4663
:1075800099469246044600F124080168880604D50D
:10759000E06921F01001216000E00120A84201DD36
:1075A000471B00E00027A1697A1902EB0900081ABD
:1075B000A0612078C00602D42046FFF721FE0026F5
:1075C00008E0D4E901211AF806009047206A401C1F
:1075D000761C20624E45F4DB2078C0060AD5204692
:1075E000FFF70EFE06E0D4E9012130209047206A23
:1075F000401C2062381EA7F10107F4DC07E0D4E943
:10760000012118F805009047206A401C2062281EBE
:10761000A5F10105F3DC2046FFF708FE20780006FF
:1076200002D50220BDE8F0870120FBE701694A1C72
:1076300002610878704700B58FB0CDE901310021B3
:10764000059105497944CDE9031011466846FFF7D5
:1076500063FE0FB000BD0000E5FFFFFF0A6802F8FF
:10766000010B0A60704710B5436913B1AFF3008096
:1076700001E0FFF7ECFD012010BD127800F12401BC
:107680000A7000224A700122EDE711684FF0FF32C4
:10769000E9E710B5203AC0F00B80B1E81850203A65
:1076A000A0E81850B1E81850A0E81850BFF4F5AFA2
:1076B0005FEA027C24BFB1E81850A0E8185044BF2C
:1076C00018C918C0BDE810405FEA827C24BF51F899
:1076D000043B40F8043B08BF7047D20728BF31F88D
:1076E000023B48BF11F8012B28BF20F8023B48BFDE
:1076F00000F8012B7047754600F02CF8AE460500E7
:107700006946534620F00700854618B020B5FFF7BC
:1077100051FDBDE820404FF000064FF000074FF04C
:1077200000084FF0000B21F00701AC46ACE8C0099F
:10773000ACE8C009ACE8C009ACE8C0098D467047A8
:1077400010B50446AFF300802046BDE81040FFF7B7
:107750001CBD000000487047B804002070470000BE
:1077600001491820ABBEFEE72600020000B585B037
:107770004FF4004000F034FC1B4800F04DF80020AE
:10778000009001208DF804008DF805004FF4602072
:1077900002900020039001208DF8100069461248E5
:1077A00000F07CF80723012205210F4800F09EF825
:1077B00001210D4800F025F801210B4800F016F8D2
:1077C000094800F0EFF800BF074800F05DF8002816
:1077D000FAD1054800F0F6F800BF034800F04AF877
:1077E0000028FAD105B000BD0024014021B1826813
:1077F00042F00102826003E0826822F001028260AE
:10780000704721B1826842F48072826003E082682E
:1078100022F480728260704710B504461248844298
:1078200008D10121401500F017FC0021601500F07F
:1078300013FC17E00D48844208D10121001500F027
:107840000BFC0021201500F007FC0BE008488442E7
:1078500008D10121C80300F0FFFB00214FF40040D4
:1078600000F0FAFB10BD0000002401400028014098
:10787000003C0140014600208A6802F004020AB17F
:10788000012000E000207047014600208A6802F0D5
:1078900008020AB1012000E00020704730B502461E
:1078A0000020002350680F4C20400D790C6844EAFA
:1078B00005242043506090680B4C2040D1E90254CD
:1078C0002C434D7944EA450420439060D06A20F46B
:1078D00070000C7C641EE4B2234340EA0350D06283
:1078E00030BD0000FFFEF0FFFDF7F1FFF0B50446EC
:1078F0000D4600200021092D11DDE068A5F10A06E2
:1079000006EB4607072606FA07F18843A5F10A06A3
:1079100006EB460603FA06F10843E0600CE0206936
:1079200005EB4507072606FA07F1884305EB4506F0
:1079300003FA06F108432061072A0FDA606B561E2E
:1079400006EB86071F2606FA07F18843561E06EB4C
:10795000860605FA06F10843606322E00D2A0FDA75
:10796000206BD61F06EB86071F2606FA07F1884311
:10797000D61F06EB860605FA06F10843206310E0E1
:10798000E06AA2F10D0606EB86071F2606FA07F14C
:107990008843A2F10D0606EB860605FA06F10843B8
:1079A000E062F0BD816841F008018160704721B15B
:1079B000826842F4A002826003E0826822F4A0029E
:1079C00082607047816841F004018160704710B5A2
:1079D000012000F051FB002000F04EFB10BD000024
:1079E00008B5014600200090034800900098084424
:1079F00000900098008808BD006C004008B5002287
:107A00000092044A0092009A02440092009A116087
:107A100008BD0000006C004000BFFEE721B1026815
:107A200042F00102026004E002684FF6FE731A4061
:107A30000260704700B58BB00121084600F0DCFA07
:107A40000F4800F023F80F4800900F4801900020E5
:107A500002900A20039000200490802005904000AE
:107A600006908000079020200890000209900020D6
:107A70000A906946024800F0AFF80BB000BD000064
:107A8000080002404C2401408403002001684FF6A6
:107A9000FE72114001600021016041608160C1609F
:107AA0004B49884208D14A490839496841F00F01D9
:107AB000474A083A51608AE045491431884208D162
:107AC00043490839496841F0F001414A083A516098
:107AD0007DE03F492831884208D13D49083949684D
:107AE00041F470613A4A083A516070E038493C31DB
:107AF000884208D136490839496841F47041344A0E
:107B0000083A516063E032495031884208D1304927
:107B10000839496841F470212D4A083A516056E00D
:107B20002B496431884208D129490839496841F410
:107B30007001274A083A516049E025497831884266
:107B400008D123490839496841F07061204A083A50
:107B500051603CE01F49884206D1011F096841F08D
:107B60000F01021F116032E01A491431884208D116
:107B70001849091F096841F0F001164A121F1160E7
:107B800025E014492831884208D11249091F0968A3
:107B900041F470610F4A121F116018E00D493C3129
:107BA000884208D10B49091F096841F47041094A0C
:107BB000121F11600BE007495031884207D1054977
:107BC000091F096841F47021024A121F11607047B1
:107BD000080002400804024010B50022026847F67F
:107BE000F0739A430C6A8B6823430C6923434C69F6
:107BF00023438C692343CC6923434C6A23438C6A17
:107C000023431A430260CB6843600B6883604B6870
:107C1000C36010BD70472DE9F041024600250026E3
:107C2000002000230024002791F803C00CF00F056A
:107C300091F803C00CF0100CBCF1000F03D091F8C8
:107C400002C04CEA050591F800C0BCF1000F31D02C
:107C5000146800202BE04FF0010C0CFA00F3B1F88F
:107C600000C00CEA03069E4220D183004FF00F0CA7
:107C70000CFA03F7BC4305FA03FC4CEA040491F840
:107C800003C0BCF1280F06D14FF0010C0CFA00FC28
:107C9000C2F814C00AE091F803C0BCF1480F05D146
:107CA0004FF0010C0CFA00FCC2F810C0401C082870
:107CB000D1D31460B1F800C0BCF1FF0F34DD5468BB
:107CC00000202EE000F1080C4FF0010808FA0CF338
:107CD000B1F800C00CEA03069E4221D183004FF0A8
:107CE0000F0C0CFA03F7BC4305FA03FC4CEA04043E
:107CF00091F803C0BCF1280F05D100F1080C08FA77
:107D00000CF8C2F8148091F803C0BCF1480F07D1F9
:107D100000F1080C4FF0010808FA0CF8C2F81080C6
:107D2000401C0828CED35460BDE8F081F0B50A4667
:107D3000002300240021002500F00046B6F1004F8A
:107D400002D11D4EF16901E01B4E7168C0F303457D
:107D500083B200F44016B6F5401F08D121F07061DF
:107D6000154E766826F07066134F7E6012E000F4C0
:107D70008016B6F5801F06D1032606FA05F4A14346
:107D800041F0706106E0460D360103FA06F6B14394
:107D900041F0706122B1460D360103FA06F6314317
:107DA00000F00046B6F1004F02D1034EF16101E050
:107DB000014E7160F0BD000000000140024600204D
:107DC00093680B400BB1012000E000207047014692
:107DD000C86880B2704702460020D3680B400BB1E0
:107DE000012000E000207047416170470161704749
:107DF000C160704770B502460D46FF21FF23002485
:107E000009E012F8010B80EA01040748005D80EAEE
:107E100003010648035D281EA5F10106B5B2F0D1A5
:107E200043EA012070BD0000D4CE0008D4CF000882
:107E300000BFFEE710B501F017FD4FF480710F4849
:107E4000FFF7D4FF40210E48FFF7D0FF02210C4876
:107E5000FFF7CCFF4FF400710848FFF7C5FF4FF460
:107E60007A7000F0D1FE4FF400710448FFF7BEFFB6
:107E70004FF4FA7000F0C8FE10BD0000000C014085
:107E80000008014070B504464FF400511148FFF757
:107E9000ABFF01F041FC1048FFF799FF00F47F4071
:107EA00040EA040529460C48FFF7A2FF4FF4807111
:107EB0000948FFF799FF02210848FFF795FF0221C3
:107EC0000648FFF793FF4FF480710348FFF78EFFDA
:107ED00070BD000000100140000C0140000801408E
:107EE00070B504464FF400511148FFF77FFF01F0D1
:107EF00013FC1048FFF76BFF00F47F4040EA0405D5
:107F000029460C48FFF774FF4FF480710948FFF7CA
:107F10006BFF02210848FFF767FF02210648FFF7C1
:107F200065FF4FF480710348FFF760FF70BD0000EC
:107F300000100140000C01400008014000BFFEE7B6
:107F4000704710B54FF4A06000F03AF810BD000083
:107F500070B5002100230F22C47804B3154C2468A7
:107F600004F4E064C4F5E064210AC1F10403CA40EA
:107F7000447804FA03F184781440214309010E4C3B
:107F80000678A155047804F01F050124AC4005785B
:107F90006D11AD0005F1E025C5F8004109E0047858
:107FA00004F01F050124AC40044D0678761145F815
:107FB000264070BD0CED00E000E400E080E100E050
:107FC00002490143024A1160704700000000FA05AF
:107FD0000CED00E0014908627047000000000E420D
:107FE00001460020034A506820F440400843506096
:107FF000704700000010024029B1064A526902434E
:10800000044B5A6104E0034A52698243014B5A61AE
:10801000704700000010024029B1064AD2690243AD
:10802000044BDA6104E0034AD2698243014BDA610E
:10803000704700000010024029B1064A92690243CD
:10804000044B9A6104E0034A92698243014B9A61AE
:10805000704700000010024029B1064AD26802436E
:10806000044BDA6004E0034AD2688243014BDA60D1
:10807000704700000010024001490860704700008E
:108080004004424230B500210022002400232D4D3F
:108090006D6805F00C0121B1042905D0082923D110
:1080A00005E0294D056022E0274D05601FE0254DC4
:1080B0006D6805F47012234D6D6805F48034022557
:1080C00005EB92421CB9214D554305600BE01D4D57
:1080D0006D6805F400351DB11C4D5543056002E087
:1080E000194D5543056002E0174D056000BF00BF04
:1080F000144D6D6805F0F0010909154D6B5C0568BC
:10810000DD4045600F4D6D6805F4E061090A104DD2
:108110006B5C4568DD4085600A4D6D6805F4605113
:10812000C90A0B4D6B5C4568DD40C560054D6D6847
:1081300005F44041890B074D6B5CC568B5FBF3F551
:10814000056130BD0010024000127A0000093D00B8
:108150000A0000201A00002010B50146002200236A
:1081600000204A11012A02D1094C236806E0022AA4
:1081700002D1074C236A01E0054C636A01F01F023B
:10818000012494401C400CB1012000E0002010BDEF
:108190000010024000210B4A11700A4A203A82F86E
:1081A0002010012802D0042808D103E00121054A4B
:1081B000117004E00521034A117000E000BF00BF08
:1081C000704700002010024001490860704700001D
:1081D0003C0442420249096A0143014A1162704764
:1081E00000100240024909888143014A118070470A
:1081F000042800400348008840F01000014908802E
:108200007047000004280040034800884FF6EF71D3
:1082100008400149088070470428004001460020BA
:10822000064A12880A40D0B2044A121F12880A4035
:1082300012B108B1012000E000207047042800407E
:1082400010B50120FFF7EAFF002831D001F05CFEF5
:108250001E480068010C0C20FFF7D0FB1B4800886B
:1082600081B21020FFF7CAFB194801881420FFF7DC
:10827000C5FB4FF400611748FFF7ADFD20B10121A8
:108280001820FFF7BBFB03E000211820FFF7B6FB27
:108290000F48008820B10E480088401E0C49088015
:1082A0000D48008820B10C480088401E0A4908800B
:1082B0000220FFF7B3FF10B10220FFF793FF052064
:1082C000FFF790FF00F02AF810BD000064000020C6
:1082D00060000020000C01406A00002029B1064A1D
:1082E00012880243044B1A8004E0034A1288824336
:1082F000014B1A80704700000028004000B502467C
:10830000FFF778FFC2F3034003490880091D0A8084
:10831000FFF77AFF00BD00000828004000BF0348B7
:10832000008800F020000028F9D0704704280040A1
:10833000074800884FF6F77108400549088000BFDC
:108340000348008800F008000028F9D070470000BA
:1083500004280040704710B500F002F810BD00007E
:108360000CB50020019000903348006840F4803044
:108370003149086000BF3048006800F400300090C8
:108380000198401C0190009818B90198B0F5A06FB1
:10839000F1D12948006800F4003010B101200090AC
:1083A00001E0002000900098012843D12348006894
:1083B00040F01000214908600846006820F00300E2
:1083C00008600846006840F0020008601A484068EB
:1083D000194948600846406848600846406840F4CB
:1083E000806048600846406820F47C104860084679
:1083F000406840F4F81048600846006840F080701B
:10840000086000BF0C48006800F000700028F9D038
:108410000948406820F00300074948600846406862
:1084200040F00200486000BF0348406800F00C00C4
:108430000828F9D10CBD00000010024000200240C5
:10844000042808D14FF0E021096941F004014FF000
:10845000E022116107E04FF0E021096921F00401F9
:108460004FF0E0221161704710B51248006840F0EB
:10847000010010490860084640680F4908400D494E
:108480004860084600680D4908400A4908600846E7
:10849000006820F4802008600846406820F4FE0050
:1084A00048604FF41F008860FFF755FF04480549F6
:1084B000086010BD001002400000FFF8FFFFF6FE4C
:1084C0000070000808ED00E010B50121154800F02B
:1084D00074F8F8B10121134800F060F80120124946
:1084E0000870124800780A2805DA10480078401C05
:1084F0000E49087015E000200C49087001200C4955
:1085000008700C480078322805DA0A480078401CC8
:108510000849087005E00020064908700120064956
:10852000087010BD000400404A0000204D000020EB
:108530004B0000204E0000204C0000207FB5054677
:108540000C4601210220FFF767FDADF80850ADF899
:1085500004400020ADF80A00ADF8060001A90E485D
:1085600000F046F8012211460B4800F037F81D20B4
:108570008DF8000001208DF8010003208DF8020025
:1085800001208DF803006846FFF7E2FC0121024854
:1085900000F007F87FBD000000040040CA430282DB
:1085A000704721B1028842F00102028004E0028893
:1085B0004FF6FE731A400280704730B50246002025
:1085C00000230024158A05EA0103958905EA0104C0
:1085D00013B10CB1012000E0002030BD1AB1838935
:1085E0000B43838102E083898B43838170470000C2
:1085F000002202881D4B98420ED01D4B98420BD092
:10860000B0F1804F08D01B4B984205D01A4B9842CE
:1086100002D01A4B984204D14FF68F731A404B8800
:108620001A43174B984207D0164B984204D04FF686
:10863000FF431A40CB881A4302808B8883850B88BE
:1086400003850A4B98420BD0094B984208D00E4B39
:10865000984205D00D4B984202D00D4B984201D163
:108660000B7A03860123838270470000002C0140AF
:10867000003401400004004000080040000C0040AD
:108680000010004000140040004001400044014040
:108690000048014010B520211F4800F05EF8012875
:1086A00015D11E480078C82802DB00201B4908703D
:1086B0001949091D0988CAB218490878411C174B85
:1086C000197017490A5400201649087023E0402108
:1086D000114800F042F801281DD140210E4800F059
:1086E00027F80E4800781049097888420ADA0B49C1
:1086F0000878411C094A11700949095C064A121D93
:10870000118008E080210948FFF76EFB0020034933
:1087100008700549087010BD003801405000002065
:10872000980300204F000020510000200008014065
:1087300001F40072B2F5007F00D100BFCA4302808D
:10874000704721B1828942F40052828104E082891B
:108750004DF6FF731A408281704702460020B1F542
:10876000007F00D100BF13880B400BB1012000E057
:1087700000207047F0B503460024002600250020A5
:1087800040F66A17B94200D100BF1846C1F342143F
:1087900001F01F06012707FA06F5012C01D10C3064
:1087A00004E0022C01D1103000E014301AB1076847
:1087B0002F43076002E00768AF430760F0BD000089
:1087C0002DE9F04786B005460E460024A24600BFBC
:1087D000A1460027B08900B100BF2F462C8A4CF675
:1087E000FF700440F08804432C82AC894EF6F310ED
:1087F0000440B08831890843718908430443AC813F
:10880000AC8A4FF6FF400440B0890443AC8201A813
:10881000FFF738FC1F48874202D1DDF810A001E0C5
:10882000DDF80CA0A88900F4004040B10AEBCA00B2
:1088300000EB0A1031684900B0FBF1F807E00AEBE1
:10884000CA0000EB0A1031688900B0FBF1F864201F
:10885000B8FBF0F004012009642101FB1089A8890C
:1088600000F4004040B1322000EBC900B0FBF1F051
:1088700000F00700044308E0322000EB09106421F7
:10888000B0FBF1F000F00F0004432C8106B0BDE80E
:10889000F08700000038014000BFFEE730380A28AA
:1088A00001D20120704700207047000010B500225F
:1088B000002014E0002107E00A4B03EB410333F8EA
:1088C00010301A444B1CD9B20A29F5DB0A23B2FB3B
:1088D000F3F3054C24F810300022431CD8B20128D1
:1088E000E8DB10BD840300202200002008B5012130
:1088F0004802FFF7A1FB00208DF803002020ADF80F
:10890000000069460748FFF786F9FEF72FFFFFF7DB
:1089100091F801210448FFF74AF801210348FFF7C5
:108920007DF808BD00080140002401400800024015
:108930002DE9F04385B004460B34A778E07840EA8F
:1089400007272579607940EA05250B3C0C226E4902
:108950002046FEF77AFD00287ED10B34607810287F
:108960007BD1C82FFCD14FF000084FF00209002046
:10897000664908804FF400616548FFF72CFA30B172
:108980006248008820F00100401C604908801021E6
:108990006048FFF720FA30B15C48008820F00800FA
:1089A00008305A4908805C4801785848008861F3CB
:1089B000CF3056490880594801885448008861F3EF
:1089C0008E1052490880084600880012ADF8000059
:1089D00008460088ADF80200072D04D04FF00308C8
:1089E0004FF001093EE0E579207A40EA05254C4840
:1089F0000580657AA07A40EA052549484580E57AF0
:108A0000207B40EA052546488580657BA07B40EABF
:108A1000052543498D71E57B207C40EA05250D72D3
:108A2000657CA07C40EA0525CD71E57C207D40EA8F
:108A300005254D720846407A022811D1012088721E
:108A400040F28A200880084600888979401A401E32
:108A500033494880084601E016E04BE040888880B2
:108A60004FF002090B3C43464A466946204601F056
:108A70000FF90546284601F023FA0020294908701D
:108A80000220294908703CE0002606E0A05D10B1F4
:108A900005B0BDE8F083701CC6B20C2EF6DB0B34BB
:108AA000607804282DD1642F2BD1012D29D11F48A6
:108AB000007800B31C48007801281CD11C480078BD
:108AC000C8B900201949087080460A20ADF8000096
:108AD0000B3C0D4801682160416861608068A060BE
:108AE000434601226946204601F0D2F80546284651
:108AF00001F0E6F905E00C48007810B901200A49B8
:108B0000087000BFC4E70000960400206C0000203D
:108B1000000C0140000801405F00002060000020C0
:108B20007A04002057000020560000203100002069
:108B30005900002010B590B0134800680190124809
:108B4000001D00680290104808300068039000245F
:108B500009E00E4901EB4400B0F8E80F0AA921F83A
:108B60001400601CC4B20C2CF3DB04A901A800F0B3
:108B70000FF8182204A90AA8FEF767FC10B9012013
:108B800010B010BD0020FBE7E8F7FF1F00600008F1
:108B900018B50022009211E002780B4B9DF80040BE
:108BA0001A5510F8012B01F8012B9DF8002001F84F
:108BB000012B9DF80020521CD2B200929DF800209B
:108BC0000C2AE9DB18BD00009604002010B504460D
:108BD0006FF00400FFF734FCE11704EB5171C1F3AF
:108BE000C701074A11701046007800EB4001C1EB45
:108BF000C0104FF6FF7101EAC0000249088010BDA5
:108C00001E0000202000002000BF411E88B2002866
:108C1000FBD170470146114A12784A434FF0E023D6
:108C20005A6100229A611A46126942F001021A61E1
:108C300000BF4FF0E022106900F001021AB100F409
:108C40008032002AF5D04FF0E022126922F00102B2
:108C50004FF0E0231A6100229A6170471E00002045
:108C600010B500F029F8012000F098FD01242246FB
:108C7000641C0B48007804FB0020C1B209A2272025
:108C800000F018FF2246641C0548007804FB002011
:108C9000C1B205A2032000F00DFF01F05DFC10BD84
:108CA000090000204D4355004465766963652049FD
:108CB00044204572726F720000200021084A00BFF4
:108CC0000BE0002004E0002302F8013B431CD8B273
:108CD0006028F8DB01F10803D9B24029F1DB7047C5
:108CE000840000207CB5FFF7E7FF052000F056FD6B
:108CF0007348007802287DD17248407A012805D156
:108D000071A21421182000F0D5FECAE06D48407A07
:108D1000022805D16DA21421202000F0CBFE59E0DD
:108D20006848007A10B16748448801E06548848843
:108D30000A20B4FBF0F52A4665A16648FEF74CFA16
:108D4000B4F57A7F05D3634A0821102000F0B2FE03
:108D500004E0604A08211C2000F0ACFE594800885D
:108D60004FF6FF71884204D15BA15A48FEF734FAEE
:108D700009E0544800880A2190FBF1F52A4654A1E5
:108D80005448FEF729FA4F480088B0F57A7F05DB92
:108D9000504A2221102000F08DFE04E04D4A22218D
:108DA0001C2000F087FE012000F0F8FC4BA21021EF
:108DB0003C2000F07FFE49A22A213C2000F07AFEF0
:108DC00047A20021142000F075FE48A23821182087
:108DD00000F070FE012000F0E1FC46480078C0B1D0
:108DE0004FF400614448FEF7F6FF38B94348008865
:108DF00020B100E037E04248007828B94FF4006124
:108E00003D48FEF7E8FF20B13EA21C21002000F003
:108E100051FE2C48807A98B13AA21C21542000F0CF
:108E200049FE2848407A00283BD101200321212314
:108E30004C22CDE900101F21102001F05FFB30E033
:108E400031A21C21482000F035FE1E48407AF8B9B6
:108E50000120032121234422CDE900101F211020ED
:108E600001F04CFB1DE01648007890B1022000F0A4
:108E700095FC27A20021084600F01CFE28A2142120
:108E8000002000F017FE29A22821042000F012FE85
:108E900007E0022000F082FC26A21821042000F046
:108EA00009FE2748007838B1012000F077FC25A2A0
:108EB0003A210A2000F0FEFD01F04EFB7CBD0000CF
:108EC000560000207A0400204F4646004F4E000016
:108ED00025326400A20400202D2D2D002500000065
:108EE000536574706F696E74000000004375727290
:108EF000656E74005F000020000C014060000020DF
:108F00005E0000204F6E00004175746F000000008D
:108F1000506C6561736520707265737300000000AA
:108F20002041646472657373696E6700202020209D
:108F30004B65790020204F66666C696E6500000005
:108F40002C000020656570720000000010B5FFF76E
:108F5000B3FE022000F022FC0AA20A21002000F049
:108F6000A9FD012000F01AFC0AA22321042000F030
:108F7000A1FD0CA23221042000F09CFD01F0ECFACE
:108F800010BD000052657365742053797374656D6C
:108F9000000000004144445220746F20636F6E66ED
:108FA00069726D00202046414E20746F206261631B
:108FB0006B00000010B5FFF77FFE022000F0EEFB13
:108FC0000AA20821002000F075FD0CA21C2100203F
:108FD00000F070FD012000F0E1FB0BA23221002027
:108FE00000F068FD01F0B8FA10BD0000526573652D
:108FF000742053797374656D0000000020202020D8
:10900000446F6E650000000020506C656173652040
:10901000526573746172740010B5FFF74DFE022043
:1090200000F0BCFB15A20421084600F043FD16A287
:109030001821042000F03EFD052000F0AFFB15488C
:10904000C07A98B11348C27A13A11448FEF7C4F845
:10905000124A2821084600F02DFD022000F09EFB58
:109060000FA230213A2000F025FD04E00DA22821B6
:10907000182000F01FFD01F06FFA10BD20486F743A
:10908000205374617274000020202044656C617963
:10909000000000007A04002025640000A2040020E3
:1090A0006D696E004F46460010B5FFF705FE0220C1
:1090B00000F074FB084A0A21202000F0FBFC074A5C
:1090C00007A10948FEF788F8074A1E21042000F08E
:1090D000F1FC01F041FA10BD6A0400206004002098
:1090E0002020205620257300A204002008B501216D
:1090F0000420FEF7A1FF03208DF8020010208DF858
:109100000300C001ADF8000069460848FEF783FD82
:109110004FF48050ADF8000014208DF8030069462C
:109120000248FEF778FD00F0B2F908BD00080140E2
:109130002DE9F04707460C4690461D46DDF8209085
:1091400000260AE000F010FA384600F0D1F900B924
:1091500005E000F014FA701CC6B2C82EF2DB00BFA6
:10916000C82E02DB0120BDE8F087B8F1020F09D15B
:10917000C4F3072000F0BCF9012803D100F0FFF987
:109180000120F0E7E0B200F0B3F9012803D100F0CC
:10919000F6F90120E7E700F0E7F947F0010000F0F9
:1091A000A7F9B8B90BE000F07BF905F8010BB9F1AC
:1091B000000F02D000F05AF901E000F049F9B9F1CE
:1091C0000000A9F1010101F0FF09ECD100F0D7F98D
:1091D0000020C8E700F0D3F90120C4E72DE9F047EB
:1091E00082460C4617469846DDE9089541E0002680
:1091F0000AE000F0B9F9504600F07AF900B905E04C
:1092000000F0BDF9701CC6B2C82EF2DB00BFC82E3C
:1092100002DB0120BDE8F087022F09D1C4F307204B
:1092200000F066F9012803D100F0A9F90120F1E767
:10923000E0B200F05DF9012803D100F0A0F90120AF
:10924000E8E711E019F8010B00F052F9012803D109
:1092500000F095F90120DDE7681EC5B2641CA8F195
:109260000100204000B901E0002DEBD100BF00F06B
:1092700086F9002DBBD10020CCE7000010B51848BE
:10928000007858B300201649087000F011FF01F073
:10929000E1F84FF400411348FEF79DFDA8B91248CC
:1092A0000078022811D111480088401C80B20F4973
:1092B000088041F27071884207DB00200B4908806A
:1092C0004FF400410748FEF791FD07480078022857
:1092D00004D04FF400410348FEF786FD10BD0000A6
:1092E0004B000020000801405600002054000020E0
:1092F00010B50548007830B100200349087000F02F
:10930000BFFDFFF7D3FA10BD4A00002010B5334867
:109310000078002860D0002030490870304800787C
:1093200002280BD12F480078401CC0B22D4908708C
:109330000A2803DB00200870294908702A480078B1
:1093400058B12A480078401CC0B228490870022849
:1093500003DB00200870244908702548007840B9D4
:109360002448007810B1FFF79FFE08E0FFF7BAFC31
:1093700005E01F480078012801D1FFF74DFE00F0FD
:109380000FF91948007840B11B48007828B11A48F5
:109390000078401E1849087002E000201249087049
:1093A0001448007820B113480078401E1149087015
:1093B0001248007818B100201049087004E00F48E6
:1093C0000078401C0D4908700D48007820B10C4809
:1093D0000078401E0A49087010BD00004C000020B3
:1093E00056000020570000203100002058000020C7
:1093F0005A00002059000020330000205E000020A9
:109400003000002002480088C0F30B0070470000C5
:109410002200002008B501210C20FEF70DFE0320DC
:109420008DF8020010208DF80300ADF800006946A9
:109430000548FEF7F0FB4FF44060ADF800006946C8
:109440000248FEF7E8FB08BD00080140000C01409F
:1094500010B5002000F04AFF012000F059FF012064
:1094600000F044FF002000F041FF10BD10B50020C7
:1094700000F03CFF002000F04BFF012000F036FF21
:10948000002000F033FF012000F042FF10BD10B5B6
:10949000012000F03DFF012000F028FF10BD00007A
:1094A00070B5012529031148FEF7A0FC00BF00207C
:1094B00000F01CFF6006040E0A20FFF7ABFB012042
:1094C00000F014FF4FF480510848FEF777FC08B114
:1094D00044F001046806050E002DE8D1002000F0DC
:1094E00005FF0A20FFF796FB204670BD00080140EB
:1094F00070B50546802400BF002000F0F7FE05EAA5
:10950000040000F005FF0A20FFF784FB012000F0B3
:10951000EDFE0A20FFF77EFB6410002CECD100204A
:1095200000F0E4FE4FF480510E48FEF75FFC0A2085
:10953000FFF770FB012000F0D9FE0A20FFF76AFB5D
:109540004FF480510748FEF739FC0646002000F032
:10955000CDFE0A20FFF75EFB0EB1012070BD00209A
:10956000FCE700000008014010B5012000F0D0FE2B
:10957000012000F0BBFE002000F0CAFE10BD10B5B7
:10958000002000F0B3FE002000F0C2FE012000F039
:10959000ADFE012000F0BCFE10BD7047704700001A
:1095A00000B50848007801280BD10748007810B1B1
:1095B000032804D100E003E000F05AF800E000BF07
:1095C00000BF00BD320000204100002010B521483E
:1095D000007830B901202049087002201F49087026
:1095E0002CE01C48007802280AD103201949087091
:1095F000012000F039FC00F03BFDFFF7DBFC1DE033
:1096000014480078012819D11548C07A032805DAD2
:109610001348C07A401C1249C87202E00020104969
:10962000C87200F0BDFF0E48C07AC0EB0010840085
:109630000C480088A04201DD0A4804800A480088DE
:1096400010B900200949088007480088401C0649D5
:10965000088010BD5A000020310000203300002097
:109660007A0400206000002046000020480000200E
:109670000B48007898B90B48007830B901200949A7
:10968000087005200649087009E00648007801289E
:1096900005D1002003490870052001490870704772
:1096A000300000205A0000207047000010B5164816
:1096B0000078022803D100201349087023E01348E2
:1096C0000088032808DB00201049088002200E498A
:1096D0000870FFF73BFC16E00D48007898B10D4884
:1096E000407A80B90848007868B90A48807A18B189
:1096F00000200849887202E001200649887200F0C3
:109700004FFFFFF7EFFA10BD5A000020460000207F
:10971000560000207A04002008B501210820FEF739
:109720008BFCFF20ADF8000003208DF80200102014
:109730008DF8030069460948FEF76DFA01210846D5
:10974000FEF77AFC01210648FEF7F0FA1820ADF882
:10975000000069460148FEF75EFA08BD000C0140B2
:10976000000230002DE9F04706460F469046994624
:10977000DDF820A034460CE03D4606E0524629467E
:10978000204600F03DFF681CC5B24D45F6DD601C6B
:10979000C4B24445F0DDBDE8F0870000014606296B
:1097A0004DD2DFE801F04C0312212E3D0822254B5B
:1097B0001A700622244B1A700822244B1A7050018A
:1097C000234A121A234B1A603AE010221D4B1A70DA
:1097D00008221D4B1A7010221C4B1A7050011E4A91
:1097E000121A1C4B1A602BE00822164B1A70164BEB
:1097F0001A70164B1A705001184A121A154B1A603B
:109800001EE00C220F4B1A7008220F4B1A700C220C
:109810000E4B1A705001124A121A0E4B1A600FE0CA
:109820003022084B1A701022074B1A701822074B6F
:109830001A7090010B4A121A064B1A6000E000BF22
:1098400000BF704700000020080000200900002031
:1098500044A6000804000020D4B200083CA9000877
:1098600054AE000804BD000808B501211C20FEF715
:10987000E3FB4220ADF8000010208DF80300032028
:109880008DF8020069461E48FEF7C5F940F2FF3028
:10989000ADF8000010208DF8030003208DF80200C1
:1098A00069461848FEF7B7F94FF40050ADF80000CC
:1098B00010208DF8030003208DF80200694612483D
:1098C000FEF7A9F901210846FEF7B6FB01210F4872
:1098D000FEF72CFA4FF40040ADF8000003208DF89D
:1098E000020010208DF8030069460548FEF793F941
:1098F0001820ADF8000069460248FEF78CF908BD53
:1099000000080140000C014000100140000230003E
:109910002DE9F04F04460D469046994600274FF03A
:10992000010B4D4507DD66B2444606F0FF086EB2F6
:109930004D4606F0FF09A8EB040046B2A9EB05006E
:109940004FFA80FA29462046099A00F059FE002E67
:1099500004DCA4EB080046B24FF0FF3B56451CDD8B
:1099600018E0002F06DD681CC5B2AAEB06003844DB
:1099700047B202E007EB0A0047B204EB0B00C4B2A7
:10998000602C01DA402D00DB06E029462046099ACA
:1099900000F036FE4445E4D11BE017E0002F07DD60
:1099A00004EB0B00C4B2A6EB0A00384447B201E056
:1099B000B81947B2681CC5B2602C01DA402D00DB33
:1099C00006E029462046099A00F01AFE4D45E5D1E9
:1099D00000BFBDE8F08F00002DE9F04706460F46B6
:1099E000924630480068304909780AFB0109002591
:1099F00051E099F80080002444E0072C16DC08F0C0
:109A0000800038B17A19D1B23219D0B2012200F0F7
:109A1000F7FD06E07A19D1B23219D0B2002200F077
:109A2000EFFD4FEA48604FEA106826E009F10100B7
:109A3000814690F8008008241AE008F0800038B1D0
:109A40007A19D1B23219D0B2012200F0D9FD06E064
:109A50007A19D1B23219D0B2002200F0D1FD4FEA0A
:109A600048604FEA1068602C00DD05E0601CC4B25D
:109A70000E4800788442E0DB00BF602C00DD05E08A
:109A8000601CC4B2094800788442B6DB00BF09F10B
:109A90000109681CC5B2064800788542A9DBBDE80B
:109AA000F0870000040000200000002008000020D3
:109AB0000900002070B505460E46144615E00D4815
:109AC00000782844602800DD12E00B48007830441C
:109AD000402800DD0CE0227831462846FFF77CFF65
:109AE000044800782844C5B2641C20780028E6D1D8
:109AF00000BF70BD08000020090000205748006822
:109B00005749B0FBF1F0C5B22846FFF75FF8FEF702
:109B100018FA01214FF0C050FEF77EFA0120FEF73F
:109B200059FAFFF7E3FA4D4800684E49B0FBF1F0EF
:109B3000401E85B229466320FEF700FD00F022FC9E
:109B4000FEF7D4FEFFF766FCFEF774F9E220FEF79D
:109B500099F9E020FEF796F9A220FEF793F9A020EC
:109B6000FEF790F9C020FEF78DF9AC20FEF78AF9D8
:109B7000A620FEF787F9A420FEF784F92C20FEF733
:109B800081F92E20FEF77EF92F20FEF77BF92520A4
:109B9000FEF778F98120FEF775F93F20FEF772F99C
:109BA000D520FEF76FF90020FEF76CF9D220FEF702
:109BB00069F90020FEF766F94020FEF763F9B0204E
:109BC000FEF760F91020FEF75DF90020FEF75AF964
:109BD000AF20FEF757F94FF400412348FEF704F990
:109BE000FEF7A8FF18B9FFF73BF800BFFEE71F49D3
:109BF0001F48FDF756FC1FA11D48FDF714FC044645
:109C000034B1211D1C48FDF74CFC641E002020705F
:109C1000FFF74AFA00F0B2F800F08AF94FF4006159
:109C20001648FEF7E1F84FF480611448FEF7DCF8BF
:109C300010210D48FEF7D8F80420114908700020C3
:109C400010490870104908701049088005E0FFF7B6
:109C50004FFBFFF713FBFFF759FBF8E770000020FD
:109C600040420F00A08601000008014020FA0108D0
:109C70006A0400205645520060040020000C014098
:109C8000590000205F0000205A0000205C000020E6
:109C90002DE9F04704460F4690469946B9F1000F6A
:109CA00007D0207B40F08001217384F80D900E25B1
:109CB00030E0207B04281AD10D254FEA4860020EBF
:109CC00029466D1C625400260EE037F81600021279
:109CD0002846691CCDB2225417F816202846691C64
:109CE000CDB22254701CC6B24645EEDB12E0207B9A
:109CF000052802D0207B10280CD10D25002607E076
:109D000017F816202846691CCDB22254701CC6B222
:109D10004645F5DB29462046FEF76CF882464FEAB9
:109D20002A206055611981F801A0A81CC0B2BDE8C5
:109D3000F08770B505460C4620780F281ADD20788C
:109D4000284410F8026C2078284410F8010C40EAEE
:109D500006262078801E81B22846FEF74BF8B042D6
:109D600005D1002020702846FEF7E2FD04E0002027
:109D7000207001E00020207070BD000038B50E2476
:109D800000BF402CFDDC1C4B01220021AE200094C2
:109D9000FFF7CEF9012802D11849087002E000202F
:109DA00016490870A01E81B21348FEF723F8124925
:109DB000898988421AD0104B01224021AE2000949C
:109DC000FFF7B6F9012802D10C49087002E0002023
:109DD0000A490870A01E81B20748FEF70BF8064931
:109DE0008989884202D0012000F03EF822460249CB
:109DF0000348FDF77AFB38BD7A0400202C000020D0
:109E00008804002010B5FFF7FDFA044640F63C70C8
:109E1000844203DD00201349087021E040F64850D9
:109E2000844203DD01200F49087019E040F68C20C0
:109E3000844203DD02200B49087011E040F26C708F
:109E4000844203DD03200749087009E0B4F5AF7FC1
:109E500003DD04200349087002E005200149087071
:109E600010BD00003900002010B504460020034951
:109E700088720320C87200F093FB10BD7A040020A2
:109E800010B580210A48FDF7A6FF80B9094800787F
:109E9000401CC0B207490870022808DB0020087087
:109EA0000548007818B104490448FFF742FF10BD87
:109EB000000801404F0000205000002098030020BF
:109EC00010B5044600200A4908700A480470802131
:109ED0000948FDF78BFF0020084908700878411CED
:109EE000064A11700649095C064A118010BD00003F
:109EF0004F000020510000200008014050000020C9
:109F0000980300200438014007480088074908608A
:109F100008460088000408600348001D008809689E
:109F20000844024908607047182800406400002077
:109F300070B500260420FDF753FD012832D0012121
:109F40004FF0C050FEF768F80120FEF743F8FDF728
:109F50003EFD0120FEF71EF900BF4120FEF7FCF890
:109F60000028FAD04FF48070FEF734F90120FEF794
:109F70002BF9FEF7D3F9FEF7DBF901210846FEF7CE
:109F8000ADF9FEF7CBF9FEF735F947F6FF70FEF7AE
:109F9000B5F9FEF7C3F9FEF737F901210420FDF703
:109FA0002DFD07E0FEF7C4F901210846FEF796F9FA
:109FB000FEF7B4F9FFF7A8FF0C20FDF711FD0646E8
:109FC0001020FDF70DFD40EA06461420FDF708FDC0
:109FD00004461820FDF704FD054604B955B3194899
:109FE000C07A38B34DB118480068801B1549C97A4A
:109FF000C1EB0111C0EB810403E013480068801B32
:10A00000241A002C03DA00201049088001E00F49CF
:10A010000C800C48C07AC0EB00100C490988B1EBE9
:10A02000800F0ADD0748C07AC0EB001080000749A6
:10A03000088002E000200549088000F009F80020AF
:10A0400070BD00007A040020640000206000002041
:10A0500008B503208DF8000000208DF801008DF870
:10A06000020001208DF803006846FDF771FF08BD6E
:10A0700010B501214FF0C050FDF7CEFF0120FDF7D4
:10A08000A9FFFDF7A4FC00210120FEF727F9FEF748
:10A0900045F90020FEF798F80020FEF77BF8002035
:10A0A000FDF798FF00214FF0C050FDF7B5FF10BD40
:10A0B00010B5FFF7A7FE72480078062879D2DFE8CE
:10A0C00000F0034E5C6A79876E480078002845D11D
:10A0D0006D48007818B900206C4908703EE06C4863
:10A0E000006800283AD06A48006803282FD96848D9
:10A0F0000068B0F5967F2AD26348007863490870FB
:10A100000846007818B308460078062813D2DFE81E
:10A1100000F0120C0903060FFFF758FA0CE0FFF7E6
:10A120003DFA09E0FFF7C2FA06E0FFF736FA03E06E
:10A13000FFF7BAFA00E000BF00BF4FF400415548F6
:10A14000FDF752FE00205449088054490880002041
:10A15000534908704E4908605249087047E0494821
:10A160000078012808D148480078012804D14848DF
:10A170000068401C4649086039E0424800780228DF
:10A1800008D141480078022804D141480068401CA9
:10A190003F4908602BE03B480078032808D13A4843
:10A1A0000078032804D13A480068401C3849086008
:10A1B0001DE01BE033480078042808D132480078BD
:10A1C000042804D132480068401C314908600EE080
:10A1D0002C480078052808D12B480078052804D1A0
:10A1E0002B480068401C2A49086000E000BF00BFFF
:10A1F00024480078244908702148007821490870D3
:10A2000023480068B0F5967F15D921480068401EA4
:10A210001F49086001202249087019480078224926
:10A2200008704FF400411B48FDF7DEFD00201A497D
:10A2300008801A49088019480088401C80B21749D4
:10A24000088041F27071884209DB002013490880C0
:10A2500016480078032802D00020144908701448DA
:10A26000008860B113480088401C80B21149088002
:10A27000B0F5FA7F03DB002008800D49088010BD8F
:10A280003900002037000020380000204000002066
:10A290003C00002000080140540000205C00002029
:10A2A0003200002036000020410000205A0000202B
:10A2B00046000020480000200848007860B10020D7
:10A2C000064908700648C07AC0EB001080000549B6
:10A2D00008803C2004490880704700006800002086
:10A2E0007A040020600000206A00002010B50446B7
:10A2F0002CB14FF400610548FDF778FD04E04FF400
:10A3000000610248FDF770FD10BD0000000801402B
:10A3100010B504462CB14FF480510548FDF766FD99
:10A3200004E04FF480510248FDF75EFD10BD0000CF
:10A330000008014010B50120064908700648008851
:10A3400038B94FF400610548FDF750FD012004497C
:10A35000087010BD5F00002060000020000C01406C
:10A360006800002010B50020044908704FF4006117
:10A370000348FDF739FDFFF79FFF10BD5F00002088
:10A38000000C014000B587B0012144F20400FDF744
:10A3900053FE03208DF81A0010208DF81B0080203A
:10A3A000ADF8180006A92948FDF735FC03208DF803
:10A3B0001A0018208DF81B004FF40070ADF818003B
:10A3C00006A92248FDF727FC48208DF81B004FF412
:10A3D0008060ADF8180006A91C48FDF71CFC4FF47E
:10A3E000964002900020ADF80C00ADF80E00ADF8DC
:10A3F0001000ADF814000C20ADF8120002A91448AA
:10A40000FEF7DEF9012240F225511148FEF7B2F9BC
:10A41000012240F226610E48FEF7ACF901210C48FA
:10A42000FEF78FF925208DF8040000208DF8050037
:10A430008DF8060001208DF8070001A8FDF788FDC2
:10A4400080210248FDF7D0FC07B000BD00080140A4
:10A450000038014010B525480078022809D1244869
:10A46000407A012805D0224800884FF6FF718842C3
:10A4700002D1FFF777FF1BE01D48007A10B11C489E
:10A48000448801E01A48848819480088A04203DC07
:10A490001748407A022802D1FFF74CFF08E0144821
:10A4A000008813498979611A884201DAFFF75AFF57
:10A4B0000E480078022803D10D48407A012804D1C3
:10A4C00010210C48FDF790FC0EE00948807A10B985
:10A4D0000948008820B110210648FDF787FC03E0F9
:10A4E00010210448FDF780FC10BD0000560000203C
:10A4F0007A040020000801406A0000202DE9F8439A
:10A5000005460E4617469846DDE9084933463A4661
:10A51000314628460094FFF7FBF943462A46314668
:10A5200028460094FFF7F4F943463A464146284648
:10A530000094FFF7EDF943463A4631463846009419
:10A54000FFF7E6F943463A4631462846CDF80090F3
:10A55000FFF708F9BDE8F88370B5002500240F4E19
:10A5600000BF17E0B02141EAE400FDF78BFC1120A9
:10A57000FDF788FC0220FDF785FC002505E016F8B4
:10A58000010BFDF7ADFC681CC5B2602DF7DB04F1D3
:10A590000800C4B2402CE5DD70BD0000840000203E
:10A5A0001CB50E24A01E81B21348FDF723FC1249EE
:10A5B00088810846102301220021CDE90004AE2045
:10A5C000FEF70CFE012802D10C49087002E00020C1
:10A5D0000A4908700848102301224021CDE90004EF
:10A5E000AE20FEF7FBFD012802D10449087002E00D
:10A5F0000020024908701CBD7A0400202C000020B5
:10A6000070B5034601F007060125B540ECB2CD1048
:10A6100005EB45050A4E06EB4515E85C012A01D11C
:10A62000204305E00AB9A04302E0022A00D16040BD
:10A63000CD1005EB4505024E06EB4515E85470BDFF
:10A6400084000020000000000000000020202020E6
:10A650002000200048484800000000005050F850FA
:10A66000F85050002078A07028F02000C0C81020BA
:10A67000409818006090A040A890680060204000BA
:10A68000000000001020404040201000402010102A
:10A6900010204000005020F820500000002020F83A
:10A6A000202000000000000000602040000000F8B2
:10A6B00000000000000000000060600000081020A2
:10A6C00040800000708898A8C88870002060202012
:10A6D00020207000708808304080F80070880830B2
:10A6E0000888700010305090F8101000F880F008C2
:10A6F00008887000304080F088887000F8081020CA
:10A700004040400070888870888870007088887821
:10A710000810600000606000606000000000606081
:10A720000060204010204080402010000000F80011
:10A73000F800000080402010204080007088081041
:10A740002000200070880868A8A87000708888F829
:10A7500088888800F08888F08888F0007088808079
:10A7600080887000E09088888890E000F88080F011
:10A770008080F800F88080F0808080007088808081
:10A7800098887800888888F8888888007020202039
:10A790002020700038101010109060008890A0C029
:10A7A000A0908800808080808080F80088D8A8A849
:10A7B000888888008888C8A89888880070888888D1
:10A7C00088887000F08888F0808080007088888891
:10A7D000A8906800F08888F0A09088007088807049
:10A7E00008887000F8202020202020008888888891
:10A7F000888870008888888888502000888888A881
:10A80000A8A85000888850205088880088888850E0
:10A8100020202000F80810204080F80070404040C0
:10A8200040407000008040201008000070101010A0
:10A830001010700020508800000000000000000090
:10A84000000000F840201000000000000000700828
:10A85000788878008080B0C88888F0000000708018
:10A8600080887000080868988888780000007088E0
:10A87000F8807000304840E0404040000000788898
:10A88000887808708080B0C88888880020006020A0
:10A89000202070001000301010109060808090A078
:10A8A000C0A0900060202020202070000000D0A8D0
:10A8B000888888000000B0C88888880000007088F8
:10A8C000888870000000F08888F080800000788818
:10A8D000887808080000B0C8808080000000788078
:10A8E0007008F0004040E040404830000000888898
:10A8F00088986800000088888850200000008888B8
:10A90000A8A85000000088502050880000008888C7
:10A91000887808700000F8102040F80010202040CF
:10A920002020100020202020202020004020201067
:10A93000202040006890000000000000000000009F
:10A9400000000000183C3C1818001800666624003F
:10A95000000000006C6CFE6CFE6C6C00183E603CED
:10A96000067C180000C6CC183066C600386C3876F5
:10A97000DCCC760018183000000000000C183030D5
:10A9800030180C0030180C0C0C18300000663CFF1E
:10A990003C6600000018187E181800000000000037
:10A9A000001818300000007E0000000000000000C9
:10A9B00000181800060C183060C08000386CC6C63D
:10A9C000C66C38001838181818187E007CC6061C8B
:10A9D0003066FE007CC6063C06C67C001C3C6CCC87
:10A9E000FE0C1E00FEC0C0FC06C67C003860C0FC29
:10A9F000C6C67C00FEC60C18303030007CC6C67C53
:10AA0000C6C67C007CC6C67E060C780000181800FE
:10AA1000001818000018180000181830060C18301C
:10AA2000180C060000007E00007E00006030180C4C
:10AA3000183060007CC60C18180018007CC6DEDEDA
:10AA4000DEC07800386CC6FEC6C6C600FC66667CF2
:10AA50006666FC003C66C0C0C0663C00F86C66667A
:10AA6000666CF800FE6268786862FE00FE626878D4
:10AA70006860F0003C66C0C0CE663A00C6C6C6FE3E
:10AA8000C6C6C6003C18181818183C001E0C0C0C42
:10AA9000CCCC7800E6666C786C66E600F0606060AE
:10AAA0006266FE00C6EEFEFED6C6C600C6E6F6DE4E
:10AAB000CEC6C6007CC6C6C6C6C67C00FC66667C22
:10AAC0006060F0007CC6C6C6C6CE7C0EFC66667CA6
:10AAD0006C66E6003C6630180C663C007E7E5A18B8
:10AAE00018183C00C6C6C6C6C6C67C00C6C6C6C6C2
:10AAF000C66C3800C6C6C6D6D6FE6C00C6C66C3854
:10AB00006CC6C6006666663C18183C00FEC68C180B
:10AB10003266FE003C30303030303C00C0603018CF
:10AB20000C0602003C0C0C0C0C0C3C0010386CC6E3
:10AB30000000000000000000000000FF30180C00C2
:10AB4000000000000000780C7CCC7600E0607C66A1
:10AB50006666DC0000007CC6C0C67C001C0C7CCC99
:10AB6000CCCC760000007CC6FEC07C003C6660F861
:10AB70006060F000000076CCCC7C0CF8E0606C7675
:10AB80006666E6001800381818183C00060006062D
:10AB90000666663CE060666C786CE600381818184B
:10ABA00018183C000000ECFED6D6D6000000DC668B
:10ABB0006666660000007CC6C6C67C000000DC66D7
:10ABC000667C60F0000076CCCC7C0C1E0000DC764D
:10ABD0006060F00000007EC07C06FC003030FC307D
:10ABE00030361C000000CCCCCCCC76000000C6C6B1
:10ABF000C66C38000000C6D6D6FE6C000000C66CDD
:10AC0000386CC6000000C6C6C67E06FC00007E4C3E
:10AC100018327E000E18187018180E001818181820
:10AC2000181818007018180E1818700076DC00003C
:10AC3000000000000C100000000000006010000088
:10AC4000000000007C82000000000000C600000040
:10AC500000000000728C00000000000000003818A6
:10AC600018183C00386C6C7866666CC018003C663E
:10AC70007E6666003000780C7CCC76001E78989E4C
:10AC8000F8989E007C6666F666667C00F0607C66DE
:10AC9000667C60F00000CC327EB0EC006830580C6E
:10ACA0007EC67C0070303C363C3078003A6CCED6A4
:10ACB000E66CB80000027CCED6E67C8000007CC644
:10ACC000FEC6C6000000FE607C60FE0000003C186E
:10ACD00018183C0000007CC6C6C67C000000C6C632
:10ACE000C6C67C000000E6F6DECEC60018001818C6
:10ACF0003C3C18003000303060C67C000C10000076
:10AD00000000000060100000000000003844000057
:10AD100000000000C600000000000000728C00006F
:10AD20000000000000000000000000100000000013
:10AD30000000000000107CD0D0D67C101C30307891
:10AD400030325C00000044382838440044287C102D
:10AD50007C10100030303000303030003840304847
:10AD600030087000C6000000000000007E425A5EFD
:10AD70005A427E0038043C443800000000366CD84B
:10AD80006C3600000000007C040400000000007C21
:10AD9000000000007C4454444C547C007C000000C3
:10ADA00000000000304830000000000010107C104F
:10ADB00010007C0060902040F0000000E010601067
:10ADC000E00000000E182000000000000000666691
:10ADD00066667CC07ED4D47414143E000000001853
:10ADE0001800000040C04040E00000003C6666667D
:10ADF0003C00000000D86C366CD80000848890A419
:10AE00004C941E04848890AC5284081EC0204024B8
:10AE1000CC141E0400663C183C6600000018007E3E
:10AE200000180000103070FC70301000203038FC2A
:10AE300038302000002070F820200000002020F88A
:10AE40007020000000082868F86020000606060C44
:10AE50008CD87830000000000000000000000000E6
:10AE60000030787878303000303000000066666658
:10AE70002400000000000000006C6CFE6C6C6CFE96
:10AE80006C6C000030307CC0C0780C0CF8303000A6
:10AE9000000000C4CC183060CC8C00000070D8D802
:10AEA00070FADECCDC76000000303030600000004C
:10AEB00000000000000C183060606030180C0000CA
:10AEC000006030180C0C0C183060000000000066A8
:10AED0003CFF3C660000000000000018187E1818B7
:10AEE0000000000000000000000000003838600092
:10AEF0000000000000FE0000000000000000000054
:10AF00000000000038380000000002060C18306015
:10AF1000C0800000007CC6CEDED6F6E6C67C00000F
:10AF2000001030F03030303030FC00000078CCCCF5
:10AF30000C183060CCFC00000078CC0C0C380C0CE9
:10AF4000CC780000000C1C3C6CCCFE0C0C1E0000ED
:10AF500000FCC0C0C0F80C0CCC780000003860C009
:10AF6000C0F8CCCCCC78000000FEC6C6060C183069
:10AF7000303000000078CCCCEC78DCCCCC78000011
:10AF80000078CCCCCC7C1818307000000000003861
:10AF90003800003838000000000000383800003861
:10AFA00038183000000C183060C06030180C0000F9
:10AFB000000000007E007E000000000000603018ED
:10AFC0000C060C18306000000078CC0C18303000F3
:10AFD00030300000007CC6C6DEDEDEC0C07C000073
:10AFE000003078CCCCCCFCCCCCCC000000FC66662D
:10AFF000667C666666FC0000003C66C6C0C0C0C6D3
:10B00000663C000000F86C66666666666CF80000D8
:10B0100000FE6260647C646062FE000000FE6662A6
:10B02000647C646060F00000003C66C6C0C0CEC6B0
:10B03000663E000000CCCCCCCCFCCCCCCCCC000010
:10B04000007830303030303030780000001E0C0C8A
:10B050000C0CCCCCCC78000000E6666C6C786C6C88
:10B0600066E6000000F060606060626666FE0000F8
:10B0700000C6EEFEFED6C6C6C6C6000000C6C6E6C0
:10B08000F6FEDECEC6C6000000386CC6C6C6C6C612
:10B090006C38000000FC6666667C606060F0000052
:10B0A00000386CC6C6C6CEDE7C0C1E0000FC666690
:10B0B000667C6C6666E600000078CCCCC07018CC6C
:10B0C000CC78000000FCB4303030303030780000F4
:10B0D00000CCCCCCCCCCCCCCCC78000000CCCCCC34
:10B0E000CCCCCCCC7830000000C6C6C6C6D6D66C58
:10B0F0006C6C000000CCCCCC783078CCCCCC000090
:10B1000000CCCCCCCC7830303078000000FECE982B
:10B1100018306062C6FE0000003C30303030303005
:10B12000303C0000000080C06030180C06020000B7
:10B13000003C0C0C0C0C0C0C0C3C000010386CC6C9
:10B1400000000000000000000000000000000000FF
:10B150000000FF0030301800000000000000000078
:10B1600000000000780C7CCCCC76000000E0606031
:10B170007C66666666DC00000000000078CCC0C01B
:10B18000CC780000001C0C0C7CCCCCCCCC76000025
:10B190000000000078CCFCC0CC78000000386C6067
:10B1A00060F8606060F000000000000076CCCCCC5D
:10B1B0007C0CCC7800E060606C76666666E6000029
:10B1C0000018180078181818187E0000000C0C00E1
:10B1D0003C0C0C0C0CCCCC7800E06060666C786C9D
:10B1E00066E600000078181818181818187E000075
:10B1F00000000000FCD6D6D6D6C600000000000035
:10B20000F8CCCCCCCCCC00000000000078CCCCCC6E
:10B21000CC78000000000000DC666666667C60F0AA
:10B220000000000076CCCCCCCC7C0C1E00000000D2
:10B23000EC6E766060F000000000000078CC6018D2
:10B24000CC78000000002060FC6060606C3800007A
:10B2500000000000CCCCCCCCCC760000000000007C
:10B26000CCCCCCCC7830000000000000C6C6D6D6CE
:10B270006C6C000000000000C66C38386CC6000022
:10B2800000000000666666663C0C18F000000000D6
:10B29000FC8C1860C4FC0000001C303060C06030C2
:10B2A000301C000000181818180018181818000092
:10B2B00000E03030180C183030E000000073DACEB7
:10B2C000000000000000000000000010386CC6C63E
:10B2D000FE00000000000000000000000000000070
:10B2E000000000000000183C3C3C1818180018181A
:10B2F00000000000006666662400000000000000F8
:10B30000000000000000006C6CFE6C6C6CFE6C6C4D
:10B310000000000018187CC6C2C07C060686C67CE9
:10B320001818000000000000C2C60C183060C68665
:10B33000000000000000386C6C3876DCCCCCCC7699
:10B34000000000000030303060000000000000000D
:10B350000000000000000C18303030303030180C85
:10B3600000000000000030180C0C0C0C0C0C183005
:10B37000000000000000000000663CFF3C6600008A
:10B3800000000000000000000018187E18180000DF
:10B390000000000000000000000000000018181865
:10B3A0003000000000000000000000FE000000006F
:10B3B000000000000000000000000000000018185D
:10B3C000000000000000000002060C183060C08081
:10B3D000000000000000386CC6C6C6C6C6C66C3881
:10B3E0000000000000001838781818181818187E87
:10B3F0000000000000007CC6060C183060C0C6FECD
:10B400000000000000007CC606063C060606C67C5E
:10B410000000000000000C1C3C6CCCFE0C0C0C1E50
:10B42000000000000000FEC0C0C0FC060606C67C8E
:10B430000000000000003860C0C0FCC6C6C6C67C64
:10B44000000000000000FEC606060C183030303048
:10B450000000000000007CC6C6C67CC6C6C6C67C0E
:10B460000000000000007CC6C6C67E0606060C78FA
:10B47000000000000000000018180000001818006C
:10B48000000000000000000018180000001818302C
:10B4900000000000000000060C18306030180C0698
:10B4A0000000000000000000007E00007E000000A0
:10B4B000000000000000006030180C060C1830601E
:10B4C0000000000000007CC6C60C181818001818F0
:10B4D000000000000000007CC6C6DEDEDEDCC07CB2
:10B4E00000000000000010386CC6C6FEC6C6C6C606
:10B4F000000000000000FC6666667C66666666FC0E
:10B500000000000000003C66C2C0C0C0C0C2663C73
:10B51000000000000000F86C6666666666666CF8FF
:10B52000000000000000FE6662687868606266FEE7
:10B53000000000000000FE6662687868606060F0ED
:10B540000000000000003C66C2C0C0DEC6C6663A0D
:10B55000000000000000C6C6C6C6FEC6C6C6C6C6F7
:10B560000000000000003C18181818181818183CA3
:10B570000000000000001E0C0C0C0C0CCCCCCC7895
:10B58000000000000000E666666C78786C6666E68F
:10B59000000000000000F06060606060606266FEB5
:10B5A000000000000000C6EEFEFED6C6C6C6C6C637
:10B5B000000000000000C6E6F6FEDECEC6C6C6C627
:10B5C0000000000000007CC6C6C6C6C6C6C6C67C53
:10B5D000000000000000FC6666667C60606060F051
:10B5E0000000000000007CC6C6C6C6C6C6D6DE7C0B
:10B5F0000C0E00000000FC6666667C6C666666E603
:10B600000000000000007CC6C660380C06C6C67C80
:10B610000000000000007E7E5A1818181818183C08
:10B62000000000000000C6C6C6C6C6C6C6C6C67CA8
:10B63000000000000000C6C6C6C6C6C6C66C3810EC
:10B64000000000000000C6C6C6C6D6D6D6FEEE6C08
:10B65000000000000000C6C66C7C38387C6CC6C692
:10B66000000000000000666666663C181818183C6A
:10B67000000000000000FEC6860C183060C2C6FE46
:10B680000000000000003C30303030303030303CC2
:10B690000000000000000080C0E070381C0E0602B0
:10B6A0000000000000003C0C0C0C0C0C0C0C0C3CC2
:10B6B0000000000010386CC6000000000000000010
:10B6C000000000000000000000000000000000007A
:10B6D00000FF00000030180C000000000000000017
:10B6E000000000000000000000780C7CCCCCCC7680
:10B6F000000000000000E06060786C666666667CB2
:10B700000000000000000000007CC6C0C0C0C67C75
:10B710000000000000001C0C0C3C6CCCCCCCCC76A7
:10B720000000000000000000007CC6FEC0C0C67C17
:10B730000000000000001C363230783030303078A5
:10B7400000000000000000000076CCCCCCCCCC7C0B
:10B750000CCC78000000E060606C7666666666E699
:10B760000000000000001818003818181818183CBD
:10B770000000000000000606000E0606060606068B
:10B7800066663C000000E06060666C78786C66E697
:10B790000000000000003818181818181818183C75
:10B7A000000000000000000000ECFED6D6D6D6C691
:10B7B000000000000000000000DC66666666666649
:10B7C0000000000000000000007CC6C6C6C6C67CA3
:10B7D000000000000000000000DC66666666667C13
:10B7E0006060F000000000000076CCCCCCCCCC7CBB
:10B7F0000C0C1E000000000000DC7666606060F04B
:10B800000000000000000000007CC660380CC67C10
:10B81000000000000000103030FC30303030361CAA
:10B82000000000000000000000CCCCCCCCCCCC76DA
:10B83000000000000000000000C6C6C6C6C66C3886
:10B84000000000000000000000C6C6D6D6D6FE6C80
:10B85000000000000000000000C66C3838386CC6DC
:10B86000000000000000000000C6C6C6C6C6C67EB6
:10B87000060CF8000000000000FECC183060C6FE88
:10B880000000000000000E18181870181818180E84
:10B8900000000000000018181818181818181818B8
:10B8A000000000000000701818180E181818187002
:10B8B000000000000076DC00000000000000000036
:10B8C0000000000000001C3000000000000000002C
:10B8D00000000000000070180000000000000000E0
:10B8E000000000000010386C0000000000000000A4
:10B8F0000000000000C6C6000000000000000000BC
:10B90000000000000076DC000000000000000000E5
:10B910000000000000000000003818181818183C3B
:10B92000000000000000386C6C6C786C6666666C19
:10B9300060C00000102810007CC6C6FEC6C6C6C681
:10B94000000000000030483000780C7CCCCCCC7675
:10B950000000000000001E7AD8D8D8FED8D8DADE61
:10B96000000000000000FC666666F6F6666666FC8F
:10B97000000000000000F0607C666666667C60F097
:10B98000000000000000000000CC323E70B0B26C3D
:10B99000000000000000D060B0187CC6C6C6C67C9F
:10B9A000000000000000E06060786C6C786060F07F
:10B9B0000000000000007CC6CECED6D6E6E6C67CEF
:10B9C0000000000000000000003A44CED6E644B873
:10B9D00000000000000000386CC6C6FEC6C6C6C621
:10B9E00000000000000000FE66626878686266FE83
:10B9F000000000000000003C181818181818183C27
:10BA0000000000000000007CC6C6C6C6C6C6C67CD4
:10BA100000000000000000C6C6C6C6C6C6C6C67C7A
:10BA200000000000000000C6E6F6FEDECEC6C6C678
:10BA30000000000000001818001818183C3C3C18C2
:10BA400000000000000030300030303060C6C67C9E
:10BA5000000000001C30000000000000000000009A
:10BA6000000000007018000000000000000000004E
:10BA700000000000386C0000000000000000000022
:10BA800000000000C6C6000000000000000000002A
:10BA90000000000076DC0000000000000000000054
:10BAA0000000000000000000000000000000000096
:10BAB000183000000000000000000000000000003E
:10BAC0000000000000000010107CD0D0D0D0D67C48
:10BAD0001010000000001C30303078303030325C04
:10BAE0000000000000000000423C24243C42000012
:10BAF000000000000000663C187E18187E18181818
:10BB00000000000000001818181800001818181875
:10BB10000000000000003C6460384444380C4C785D
:10BB20000000000000C6C600000000000000000089
:10BB300000000000000000007E425A5E5A427E0073
:10BB40000000000000007008788888740000000081
:10BB5000000000000000000000366CD86C360000C9
:10BB60000000000000000000000000FC04040000D1
:10BB700000000000000000000000007C0000000049
:10BB800000000000000000007C4454444C547C0041
:10BB900000000000FE0000000000000000000000A7
:10BBA000000000000070D888D8700000000000007D
:10BBB000000000000000000010107C1010007C004D
:10BBC00000000000788C0C183060FC0000000000C1
:10BBD00000000000788C0C780C8C780000000000CD
:10BBE00000000000000E182000000000000000000F
:10BBF0000000000000000000006666666666667C65
:10BC00006060C00000007ED4D4D474141414143EB8
:10BC1000000000000000000000003838380000007C
:10BC20000000000060E060606060F0000000000064
:10BC30000000000000003C6666663C00000000005A
:10BC4000000000000000000000D86C366CD8000036
:10BC500000000000000040C0444810244C941E0422
:10BC600000000000000040C04448102C5284081E10
:10BC7000000000000000C0204428D0244C941E0482
:10BC8000000000000000000000663C183C66000058
:10BC900000000000000000001818007E00181800C6
:10BCA0000000000000000000000818387FFF7F3807
:10BCB00018080000000000000010181CFEFFFE1C09
:10BCC0001810000000000000000010387CFE38381A
:10BCD0003838000000000000000038383838FE7C9A
:10BCE000381000000000000606060616367EFE7CB0
:10BCF00030100000000000000000030306060CCC1A
:10BD00007838000000000000000000000000000083
:10BD10000000000000000000000000000000000023
:10BD20000000000000000000000000000000000013
:10BD30000000000000000000000000003800380093
:10BD4000380038003800380038003800380010005B
:10BD5000100000003800380038000000000000002B
:10BD600000000000000000000000000073807380ED
:10BD700073807380738000000000000000000000EA
:10BD800000000000000000000000000000000000B3
:10BD90000000000000000000000000000C600C60CB
:10BDA0000C6018C0FFF0FFF018C039C03180FFF000
:10BDB000FFF031807380630063000000000000002A
:10BDC0000000000000000000000006001F803FC0CF
:10BDD00076E076E076007E003F001FC007E006E0D8
:10BDE00006E076E076E03FC01F8006000600000017
:10BDF0000000000000000000000000003C187E3839
:10BE000066306630666066607EC03CC0019E01BFE1
:10BE100003B3033303330633063F0C1E0000000058
:10BE200000000000000000000000000007800FC0BC
:10BE30001CE01CE01EE00FC00F801F803F9C71FCC7
:10BE400071F870F079FC3FFE1F8C000000000000CC
:10BE50000000000000000000000000007000700002
:10BE60007000700070000000000000000000000082
:10BE700000000000000000000000000000000000C2
:10BE80000000000000000000000000000C0018008E
:10BE900018003800380070007000700070007000EA
:10BEA0007000700070003000380038001800180072
:10BEB0000C000000000000000000000060003000E6
:10BEC0003000380038001C001C001C001C001C0046
:10BED0001C001C001C001800380038003000300026
:10BEE00060000000000000000000000018001800C2
:10BEF000DB00FF001C003C00660024000000000086
:10BF00000000000000000000000000000000000031
:10BF10000000000000000000000000000000000021
:10BF200007000700070007007FF07FF07FF00700A1
:10BF300007000700070000000000000000000000EC
:10BF400000000000000000000000000000000000F1
:10BF500000000000000000000000000000000000E1
:10BF600000000000700070007000100030006000E1
:10BF700000000000000000000000000000000000C1
:10BF80000000000000000000000000007E007E00B5
:10BF90007E00000000000000000000000000000023
:10BFA0000000000000000000000000000000000091
:10BFB0000000000000000000000000000000000081
:10BFC0000000000070007000700000000000000021
:10BFD0000000000000000000000000000C000C0049
:10BFE00018001800180038003000300030006000E1
:10BFF000600060006000C000C000000000000000A1
:10C000000000000000000000000000000F003FC022
:10C0100039C070E070E070E070E070E070E070E0F7
:10C0200070E070E039C03FC00F0000000000000069
:10C0300000000000000000000000000003800380FA
:10C0400007801F803F803B80238003800380038024
:10C050000380038003800380038000000000000051
:10C060000000000000000000000000001F803FC032
:10C0700079E070E000E000E001C003C007800F003D
:10C080001E001C0038007FE07FE000000000000080
:10C090000000000000000000000000001F003F80C2
:10C0A00071C071C001C003C00F800F8001C000E0EB
:10C0B00000E070E079C03FC01F00000000000000F9
:10C0C0000000000000000000000000000380078066
:10C0D00007800F800F801B80338033806380C38094
:10C0E000FFE0FFE003800380038000000000000009
:10C0F0000000000000000000000000001FC01FC082
:10C100003800380038003F807FC071E000E000E078
:10C1100000E070E079C03FC01F0000000000000098
:10C120000000000000000000000000000F803FC081
:10C1300039E07080700077807FC079C070E070E077
:10C1400070E070E039C03FC00F0000000000000048
:10C150000000000000000000000000007FE07FE021
:10C1600000E001C003800380070007000E000E00FE
:10C170000E001C001C001C001C0000000000000041
:10C180000000000000000000000000001F803FC011
:10C1900079E070E070E039C01F801F8039C070E026
:10C1A00070E070E079E03FC01F80000000000000F8
:10C1B0000000000000000000000000000F003FC071
:10C1C00039C070E070E070E070E039E03FE01EE000
:10C1D00000E030E079C03FC01F0000000000000018
:10C1E000000000000000000000000000000000004F
:10C1F0000000000038003800380000000000000097
:10C200000000000038003800380000000000000086
:10C21000000000000000000000000000000000001E
:10C220000000000038003800380000000000000066
:10C230000000000038003800380008001800300006
:10C2400000000000000000000000000000000000EE
:10C25000002000E007E01F807C0070007E001FC00F
:10C2600007E000E0002000000000000000000000E7
:10C2700000000000000000000000000000000000BE
:10C28000000000007FE07FE07FE0000000007FE032
:10C290007FE07FE0000000000000000000000000E0
:10C2A000000000000000000000000000000000008E
:10C2B000400070007E001F8003E000E007E03F8048
:10C2C0007E00700040000000000000000000000040
:10C2D0000000000000000000000000000F803FE0B0
:10C2E00078F07070007000F001E003C00780070074
:10C2F0000700000007000700070000000000000022
:10C3000000000000000000000000000003E007F053
:10C310000F1C1C0E19CE33E63666666666666666C8
:10C3200066666666666663FE31BE380E1C1C0F3C90
:10C3300007F003E0000000000000000007C007C095
:10C3400007C00EE00EE00EE01C701C7038383FF89D
:10C350003FF87FFC701C701CE00E00000000000025
:10C360000000000000000000000000003FE03FF07F
:10C370003FF83838383838383FF03FF03FF8381C4D
:10C38000381C381C3FFC3FF83FF000000000000064
:10C3900000000000000000000000000007C01FF0C7
:10C3A0003FF83C3C7818700070007000700070001E
:10C3B00078183C3C3FF81FF007C000000000000068
:10C3C0000000000000000000000000003FE03FF01F
:10C3D0003FF83838383C381C381C381C381C381C9E
:10C3E000381C38383FF83FF03FC000000000000024
:10C3F0000000000000000000000000003FF83FF8CF
:10C400003FF83800380038003FF03FF03FF0380088
:10C41000380038003FF83FF83FF800000000000007
:10C420000000000000000000000000003FF03FF0AE
:10C430003FF03800380038003FE03FE03FE0380090
:10C4400038003800380038003800000000000000D4
:10C4500000000000000000000000000003E00FF8F2
:10C460001FFC3C1E780C7000700070FE70FE70FEA9
:10C47000380E3C1E1FFE0FFC03E000000000000011
:10C48000000000000000000000000000703870385C
:10C4900070387038703870387FF87FF87FF87038EF
:10C4A0007038703870387038703800000000000044
:10C4B0000000000000000000000000000380038076
:10C4C0000380038003800380038003800380038054
:10C4D00003800380038003800380000000000000CD
:10C4E00000000000000000000000000001C001C0CA
:10C4F00001C001C001C001C001C001C001C0E1C054
:10C50000E1C0F1C07FC07F801E000000000000007D
:10C51000000000000000000000000000383C3878F7
:10C5200038F038E039C03B803FC03FC03EE03CE0DF
:10C53000387038383838381C381C000000000000CB
:10C54000000000000000000000000000380038007B
:10C55000380038003800380038003800380038001B
:10C56000380038003FF03FF03FF0000000000000CE
:10C570000000000000000000000000007C1F7E3F63
:10C580007E3F763776377637777777777367736757
:10C5900073E773E773E771C771C70000000000001D
:10C5A0000000000000000000000000007038783833
:10C5B00078387C387E3876387738733873B871B805
:10C5C00071F870F870F870787038000000000000A2
:10C5D00000000000000000000000000007E01FF85D
:10C5E0003FFC3C3C781E700E700E700E700E700E8C
:10C5F000781E3C3C3FFC1FF807E0000000000000F4
:10C600000000000000000000000000003FE03FF0DC
:10C610003FF83878383838783FF83FF03FE0380056
:10C6200038003800380038003800000000000000F2
:10C6300000000000000000000000000007E01FF8FC
:10C640003FFC3C3C781E700E700E700E700E708EAB
:10C6500079DE3CFC3FFC1FFE07EF000600000000F7
:10C660000000000000000000000000003FE03FF07C
:10C670003FF83838383838383FF83FF03FC038E0B6
:10C6800038F0387038383838381C000000000000A6
:10C6900000000000000000000000000007C01FF0C4
:10C6A0003FF0387838383C001F800FF003F00078F6
:10C6B000703878783FF83FF00FC0000000000000AD
:10C6C0000000000000000000000000007FF07FF08C
:10C6D0007FF00700070007000700070007000700BA
:10C6E0000700070007000700070000000000000027
:10C6F00000000000000000000000000070387038EA
:10C7000070387038703870387038703870387038E9
:10C71000703878783FF03FF00FC000000000000054
:10C72000000000000000000000000000E038E07899
:10C7300070707070707038E038E038E01DC01DC057
:10C740001DC00F800F800F80070000000000000058
:10C75000000000000000000000000000E187E18709
:10C76000718E718E718E718E399C399C399C399C79
:10C770001DB81DB81E781E781E781E7800000000B7
:10C780000000000000000000000000007038703859
:10C7900038701CE01CE00FC00780078007800FC0C6
:10C7A0001CE01CE038707038703800000000000099
:10C7B000000000000000000000000000E038E03849
:10C7C000707038E038E01DC00F800F800700070050
:10C7D0000700070007000700070000000000000036
:10C7E0000000000000000000000000007FF07FF06B
:10C7F0007FF000F001E003C007800F001E003C0046
:10C800007800F000FFF0FFF0FFF0000000000000F3
:10C810000000000000000000000000003E003E009C
:10C820003E00380038003800380038003800380042
:10C830003800380038003800380038003E003E002C
:10C840003E0000000000000000000000C000C0002A
:10C850006000600060006000300030003000380090
:10C860001800180018000C000C0000000000000068
:10C87000000000000000000000000000F800F800C8
:10C88000F800380038003800380038003800380028
:10C89000380038003800380038003800F800F80058
:10C8A000F8000000000000000000000006000F007B
:10C8B0000F001F80198039C039C070E000000000EF
:10C8C0000000000000000000000000000000000068
:10C8D0000000000000000000000000000000000058
:10C8E0000000000000000000000000000000000048
:10C8F0000000000000000000000000000000FFF049
:10C90000FFF000000000000000000000E0006000F8
:10C9100030000000000000000000000000000000E7
:10C920000000000000000000000000000000000007
:10C9300000000000000000000000000000000000F7
:10C94000000000001F803FC060E003E01FE03CE00B
:10C9500070E070E071E03FE01E7000000000000039
:10C9600000000000000000000000000070007000E7
:10C970007000700077807FE078E070707070707089
:10C980007070707078E07FE0778000000000000039
:10C990000000000000000000000000000000000097
:10C9A000000000000F003FC039C070E07000700050
:10C9B000700070E039C03FC00F00000000000000B0
:10C9C0000000000000000000000000000070007087
:10C9D000007000700F703FF038F070707070707001
:10C9E0007070707038F03FF00F70000000000000B1
:10C9F0000000000000000000000000000000000037
:10CA0000000000000F003FC039C070E07FE07FE011
:10CA1000700070E039C03FC00F000000000000004F
:10CA200000000000000000000000000000F001F025
:10CA3000038003803FFC3FFC03800380038003806E
:10CA40000380038003800380038000000000000057
:10CA500000000000000000000000000000000000D6
:10CA6000000000000F703FF038F070707070707050
:10CA70007070707038F03FF01F70007070F07FE0E1
:10CA80001FC00000000000000000000070007000E7
:10CA90007000700073C07FE078F07070707070701C
:10CAA0007070707070707070707000000000000026
:10CAB0000000000000000000000000000380038070
:10CAC0000000000003800380038003800380038054
:10CAD00003800380038003800380000000000000C7
:10CAE0000000000000000000000000000380038040
:10CAF0000000000003800380038003800380038024
:10CB00000380038003800380038003800380070089
:10CB10000E00000000000000000000007000700027
:10CB20007000700070E071C073807F007F007F0034
:10CB30007B80718071C070E070E000000000000038
:10CB400000000000000000000000000003800380DF
:10CB500003800380038003800380038003800380BD
:10CB60000380038003800380038000000000000036
:10CB700000000000000000000000000000000000B5
:10CB80000000000077CF7FFF71C771C771C771C701
:10CB900071C771C771C771C771C70000000000007D
:10CBA0000000000000000000000000000000000085
:10CBB0000000000073C07FE078F0707070707070DB
:10CBC0007070707070707070707000000000000005
:10CBD0000000000000000000000000000000000055
:10CBE000000000000F803FE038E0707070707070DF
:10CBF0007070707038E03FE00F80000000000000AF
:10CC00000000000000000000000000000000000024
:10CC10000000000077807FE078E0707070707070C6
:10CC20007070707078E07FE0778070007000700046
:10CC30007000000000000000000000000000000084
:10CC4000000000000F703FF038F07070707070706E
:10CC50007070707038F03FF00F70007000700070EE
:10CC60000070000000000000000000000000000054
:10CC700000000EFC0FFC03C00380038003800380D0
:10CC80000380038003800380038000000000000015
:10CC90000000000000000000000000000000000094
:10CCA000000000001F803FC070E070007E003FC0A9
:10CCB00007E000E070E03FC01F80000000000000BF
:10CCC00000000000000000000000000000000380E1
:10CCD000038003800FF00FF0038003800380038044
:10CCE00003800380038001F000F0000000000000DA
:10CCF0000000000000000000000000000000000034
:10CD000000000000707070707070707070707070E3
:10CD10007070707078F03FF01F700000000000002D
:10CD20000000000000000000000000000000000003
:10CD3000000000007070707038E038E038E01DC00E
:10CD40001DC00F800F8007000700000000000000DA
:10CD500000000000000000000000000000000000D3
:10CD600000000000E38EE38E638C77DC76DC36D83F
:10CD700036D83EF83C781C701C70000000000000A3
:10CD800000000000000000000000000000000000A3
:10CD90000000000070E039C039C01F800F000F0094
:10CDA0000F001F8039C039C070E000000000000093
:10CDB0000000000000000000000000000000000073
:10CDC00000000000E0E0E0E071C071C071803B80D5
:10CDD0003B801B001F001F000E000E001C007C008B
:10CDE00078000000000000000000000000000000CB
:10CDF000000000007FC07FC001C0038007000E005C
:10CE00001C00380070007FC07FC0000000000000E0
:10CE100000000000000001000100400223C40FF0E8
:10CE20001FF81FF8DFFB1FF81FF80FF023C44002A4
:10CE300001000100000000000000000000000000F0
:10CE40000000000000000000000000003000300082
:10CE50003000300030003000300030003000300052
:10CE60003000300030003000300030003000300042
:10CE700030003000000000800080000113C209F083
:10CE800000F80078187B007800F809F013C2000160
:10CE90000080008000000000000000000000000092
:10CEA0000000000000000000000000000000000082
:10CEB00000000000000000007C20FFE0FFE087C0D1
:10CEC0000000000000000000000000000000000062
:10CED0000000000000C1814001C0804101C08041CC
:10CEE00000C1814001C0804100C1814000C181403A
:10CEF00001C0804101C0804100C1814000C181402A
:10CF000001C0804100C1814001C0804101C0804119
:10CF100000C1814001C0804100C1814000C1814009
:10CF200001C0804100C1814001C0804101C08041F9
:10CF300000C1814000C1814001C0804101C08041E9
:10CF400000C1814001C0804100C1814000C18140D9
:10CF500001C0804101C0804100C1814000C18140C9
:10CF600001C0804100C1814001C0804101C08041B9
:10CF700000C1814000C1814001C0804101C08041A9
:10CF800000C1814001C0804100C1814000C1814099
:10CF900001C0804100C1814001C0804101C0804189
:10CFA00000C1814001C0804100C1814000C1814079
:10CFB00001C0804101C0804100C1814000C1814069
:10CFC00001C0804100C1814001C0804101C0804159
:10CFD00000C1814000C0C101C30302C2C60607C729
:10CFE00005C5C404CC0C0DCD0FCFCE0E0ACACB0B99
:10CFF000C90908C8D81819D91BDBDA1A1EDEDF1FC9
:10D00000DD1D1CDC14D4D515D71716D6D21213D3B8
:10D0100011D1D010F03031F133F3F23236F6F73768
:10D02000F53534F43CFCFD3DFF3F3EFEFA3A3BFB58
:10D0300039F9F83828E8E929EB2B2AEAEE2E2FEF08
:10D040002DEDEC2CE42425E527E7E62622E2E32378
:10D05000E12120E0A06061A163A3A26266A6A767A8
:10D06000A56564A46CACAD6DAF6F6EAEAA6A6BAB18
:10D0700069A9A86878B8B979BB7B7ABABE7E7FBF48
:10D080007DBDBC7CB47475B577B7B67672B2B37338
:10D09000B17170B0509091519353529296565797E8
:10D0A000559594549C5C5D9D5F9F9E5E5A9A9B5BD8
:10D0B00099595898884849894B8B8A4A4E8E8F4F88
:10D0C0008D4D4C8C448485458747468682424383F8
:10D0D0004181804030FA01080000002084000000F7
:10D0E00028710008B4FA010884000020941600009A
:10D0F0004471000800000000000000000000000073
:10D10000000000000000000000000000000000001F
:10D11000000000000000000000000000000000000F
:10D1200000000000000000000000000000000000FF
:10D1300000000000000000000000000000000000EF
:020000040801F1
:10FA00005745535442524944474500000000000006
:10FA100000000000000000000000000000000000E6
:10FA200048532D312056455220312E310000000020
:10FA300000000000000000000000000000000102C3
:10FA40000304010203040607080902040608000073
:10FA500000000000000000000000000000000000A6
:10FA60000000000000000000000000000000000096
:10FA70000000000000000000000000000000000086
:10FA80000000000000000000000000000000000076
:10FA90000000000000000000000000000000000066
:10FAA00000A24A040000000000000000010203045C
:04FAB0000607080934
:04000005080070ED92
:00000001FF
